:1000000019C033C032C031C030C02FC02EC02DC087
:100010002CC02BC02AC029C028C027C027C025C09B
:1000200024C023C082C421C020C01FC01EC01DC068
:100030001CC01BC011241FBECFEFD4E0DEBFCDBF5C
:1000400014E0A0E0B1E0EEE8FBE002C005900D9204
:10005000A032B107D9F714E0A0E2B4E001C01D92CC
:10006000A733B107E1F77ED390C5CACF1F920F9295
:100070000FB60F921124EF92FF920F931F932F93BD
:100080003F934F935F936F937F938F939F93AF9320
:10009000BF93EF93FF9380912004282F2F5F20932D
:1000A00020042A3080F480E0E8E2F0E010828F5FE4
:1000B0008C33E1F780E188B980E091E090932204ED
:1000C000809321043AC3E8E2F0E0108210821082AB
:1000D0001082108280E18083233308F42EC380E0F5
:1000E00090E190838F5F8832E1F7233D08F025C3CC
:1000F000E0912104F091220490813181E280F3802B
:1001000004811581B681A7817085618552854385FB
:1001100099231CF480E388B903C0000080E188B90A
:1001200096FF03C080E388B903C0000080E188B96E
:1001300095FF03C080E388B903C0000080E188B95F
:1001400094FF03C080E388B903C0000080E188B950
:1001500093FF03C080E388B903C0000080E188B941
:1001600092FF03C080E388B903C0000080E188B932
:1001700091FF03C080E388B903C0000080E188B923
:1001800090FF03C080E388B903C0000080E188B914
:1001900033231CF480E388B903C0000080E188B9F0
:1001A000932F36FF03C080E388B903C0000080E1CD
:1001B00088B995FF03C080E388B903C0000080E1DF
:1001C00088B994FF03C080E388B903C0000080E1D0
:1001D00088B993FF03C080E388B903C0000080E1C1
:1001E00088B992FF03C080E388B903C0000080E1B2
:1001F00088B991FF03C080E388B903C0000080E1A3
:1002000088B990FF03C080E388B903C0000080E193
:1002100088B9EE201CF480E388B903C0000080E1B7
:1002200088B99E2DE6FE03C080E388B903C00000B4
:1002300080E188B995FF03C080E388B903C000005E
:1002400080E188B994FF03C080E388B903C000004F
:1002500080E188B993FF03C080E388B903C0000040
:1002600080E188B992FF03C080E388B903C0000031
:1002700080E188B991FF03C080E388B903C0000022
:1002800080E188B990FF03C080E388B903C0000013
:1002900080E188B9FF201CF480E388B903C0000026
:1002A00080E188B99F2DF6FE03C080E388B903C0C2
:1002B000000080E188B995FF03C080E388B903C0DE
:1002C000000080E188B994FF03C080E388B903C0CF
:1002D000000080E188B993FF03C080E388B903C0C0
:1002E000000080E188B992FF03C080E388B903C0B1
:1002F000000080E188B991FF03C080E388B903C0A2
:10030000000080E188B990FF03C080E388B903C092
:10031000000080E188B900231CF480E388B903C0A1
:10032000000080E188B9902F06FF03C080E388B900
:1003300003C0000080E188B995FF03C080E388B95D
:1003400003C0000080E188B994FF03C080E388B94E
:1003500003C0000080E188B993FF03C080E388B93F
:1003600003C0000080E188B992FF03C080E388B930
:1003700003C0000080E188B991FF03C080E388B921
:1003800003C0000080E188B990FF03C080E388B912
:1003900003C0000080E188B911231CF480E388B910
:1003A00003C0000080E188B9912F16FF03C080E3ED
:1003B00088B903C0000080E188B995FF03C080E3DD
:1003C00088B903C0000080E188B994FF03C080E3CE
:1003D00088B903C0000080E188B993FF03C080E3BF
:1003E00088B903C0000080E188B992FF03C080E3B0
:1003F00088B903C0000080E188B991FF03C080E3A1
:1004000088B903C0000080E188B990FF03C080E391
:1004100088B903C0000080E188B9BB231CF480E3E5
:1004200088B903C0000080E188B99B2FB6FF03C0E4
:1004300080E388B903C0000080E188B995FF03C05C
:1004400080E388B903C0000080E188B994FF03C04D
:1004500080E388B903C0000080E188B993FF03C03E
:1004600080E388B903C0000080E188B992FF03C02F
:1004700080E388B903C0000080E188B991FF03C020
:1004800080E388B903C0000080E188B990FF03C011
:1004900080E388B903C0000080E188B9AA231CF476
:1004A00080E388B903C0000080E188B99A2FA6FFD5
:1004B00003C080E388B903C0000080E188B995FFDC
:1004C00003C080E388B903C0000080E188B994FFCD
:1004D00003C080E388B903C0000080E188B993FFBE
:1004E00003C080E388B903C0000080E188B992FFAF
:1004F00003C080E388B903C0000080E188B991FFA0
:1005000003C080E388B903C0000080E188B990FF90
:1005100003C080E388B903C0000080E188B9772375
:100520001CF480E388B903C0000080E188B9972FEC
:1005300076FF03C080E388B903C0000080E188B97A
:1005400095FF03C080E388B903C0000080E188B94B
:1005500094FF03C080E388B903C0000080E188B93C
:1005600093FF03C080E388B903C0000080E188B92D
:1005700092FF03C080E388B903C0000080E188B91E
:1005800091FF03C080E388B903C0000080E188B90F
:1005900090FF03C080E388B903C0000080E188B900
:1005A00066231CF480E388B903C0000080E188B9A9
:1005B000962F66FF03C080E388B903C0000080E186
:1005C00088B995FF03C080E388B903C0000080E1CB
:1005D00088B994FF03C080E388B903C0000080E1BC
:1005E00088B993FF03C080E388B903C0000080E1AD
:1005F00088B992FF03C080E388B903C0000080E19E
:1006000088B991FF03C080E388B903C0000080E18E
:1006100088B990FF03C080E388B903C0000080E17F
:1006200088B955231CF480E388B903C0000080E139
:1006300088B9952F56FF03C080E388B903C0000036
:1006400080E188B995FF03C080E388B903C000004A
:1006500080E188B994FF03C080E388B903C000003B
:1006600080E188B993FF03C080E388B903C000002C
:1006700080E188B992FF03C080E388B903C000001D
:1006800080E188B991FF03C080E388B903C000000E
:1006900080E188B990FF03C080E388B903C00000FF
:1006A00080E188B944231CF480E388B903C00000CA
:1006B00080E188B9942F46FF03C080E388B903C066
:1006C000000080E188B995FF03C080E388B903C0CA
:1006D000000080E188B994FF03C080E388B903C0BB
:1006E000000080E188B993FF03C080E388B903C0AC
:1006F000000080E188B992FF03C080E388B903C09D
:10070000000080E188B991FF03C080E388B903C08D
:10071000000080E188B990FF03C080E388B903C07E
:10072000000080E188B980E188B920FD06C0CF01D2
:100730000C969093220480932104FF91EF91BF9136
:10074000AF919F918F917F916F915F914F913F9169
:100750002F911F910F91FF90EF900F900FBE0F9070
:100760001F9018950F931F93CF93DF9304E210E02F
:1007700080E1E80188838FEF87B98EE38AB918B8E2
:100780008FE190E099D0888180618883E5E2F0E094
:1007900080818061808327E430E08FE7F9018083E6
:1007A000A4E4B0E092E09C93E5E4F0E090838EE96D
:1007B000E90188839C93908300E0802F64E6B2D1A6
:1007C0006AE0B0D1892F805D99D1802F6AE0AAD1EB
:1007D000A9D1892F805D92D1802F6AE0A3D1892F82
:1007E000805D8CD18CE28AD188E7EAD083E1E8D0C1
:1007F00088E3E6D082E5E4D0C6D0EC01EFEF8F3F8E
:100800009E07D1F364E68ED16AE08CD1892F805D9A
:1008100075D18C2F6AE086D185D1892F805D6ED10C
:100820008C2F6AE07FD1892F805D68D18CE266D100
:10083000AAD0EC01FFEF8F3F9F07D1F364E672D19E
:100840006AE070D1892F805D59D18C2F6AE06AD11E
:1008500069D1892F805D52D18C2F6AE063D1892FB5
:10086000805D4CD18CE24AD18ED0EC018FEFCF3F2E
:10087000D807D1F38C2F64E655D16AE053D1892F84
:10088000805D3CD18C2F6AE04DD14CD1892F805DA9
:1008900035D18C2F6AE046D1892F805D2FD18DE034
:1008A0002DD18AE02BD10F5F88CF109226041092B1
:1008B00025041092270408959093C5008093C400E6
:1008C000E0ECF0E080818D7F808380818E7F80836B
:1008D000A1ECB0E08C9180688C938C918F7B8C9391
:1008E0008C9180618C938C9188608C93E2ECF0E029
:1008F00080818F7B808380818F77808380818F7ED2
:10090000808380818F7D80838081877F80838C91AD
:100910008B7F8C93808184608083808182608083E0
:1009200080818E7F8083C1DF08951F920F920FB662
:100930000F9211242F938F939F93EF93FF938091A6
:10094000C0008823B4F42091C60080912504982F1C
:100950009F5F903108F090E080912604891749F05C
:1009600080912504E7E2F4E0E80FF11D20839093E5
:100970002504FF91EF919F918F912F910F900FBEC2
:100980000F901F9018959091260480912504981738
:1009900019F4EFEFFFEF11C080912604E7E2F4E0D5
:1009A000E80FF11D9081809126048F5F803108F05F
:1009B00080E080932604E92FF0E08E2F9F2F08958A
:1009C000982FE0ECF0E0808185FFFDCF9093C6008A
:1009D00081E008951F93CF93DF93EC0188818823F2
:1009E00059F010E0EDDF882341F0219688818823BB
:1009F00019F01F5F1031B1F781E0DF91CF911F91A6
:100A000008951F93182F82958F70EEE0F4E0E80FA1
:100A1000F11D8081D5DF882351F0E12FF0E0EF70E8
:100A2000F070E25FFB4F8081CBDF811181E01F918D
:100A300008951F93182F90E068EE73E07FD064E66E
:100A400070E07CD0862F805DBBDF8823A1F0812FF2
:100A500064E668D0892F6AE065D0805DB1DF8823C5
:100A600051F0812F6AE05ED0892F805DA9DF882355
:100A700019F081E001C080E01F9108950F931F934A
:100A8000082F162F8BE19CDF8BE59ADF812F8F5F7C
:100A9000D0DF8BE395DF802F8F5FCBDF88E490DFA3
:100AA0001F910F9108958BE18BDF8BE589DF82E346
:100AB00087DF8AE485DF08951F93182F8BE180DF9D
:100AC0008BE57EDF812FB5DF8DE67ADF1F910895FC
:100AD0008BE176DF8BE574DF8EE372DF85E370DF19
:100AE0008CE66EDF08958BE16BDF8BE569DF8EE3CB
:100AF00067DF85E365DF88E663DF08951F932F9343
:100B0000809508942AE01BE01A95F1F708F02C9ADA
:100B100008F42C9886952A95B1F72A95F1F72F912C
:100B20001F910895991B79E004C0991F961708F04A
:100B3000961B881F7A95C9F78095089597FB092E13
:100B400007260AD077FD04D00CD006D000201AF476
:100B5000709561957F4F0895F6F7909581959F4F19
:100B60000895AA1BBB1B51E107C0AA1FBB1FA617F4
:100B7000B70710F0A61BB70B881F991F5A95A9F746
:0E0B800080959095BC01CD010895F894FFCFAB
:100B8E00FFFFFFFFFFFFFFFFFFFFFFFFFFFFFFFF67
:100B9E00FFFFF3FFFFFFFFFFFFFFFFFFFFFFE3FF7F
:100BAE00FFFFFFFFFFFFFFFFFFFFE3FFFFFFFFFF63
:100BBE00FFFFFFFFFFFFC7FFFFFFFFFFFFFFEFFF7F
:100BCE00FFFF83FFFFFFFFF7FFFFD7FFFFFF87FF4B
:100BDE00FFFFFFEFFFFF87FFFFFF07FFFFFFFFFF97
:100BEE00FFFFD3FFFFFE07FFFFFFFFCFFFFFE1FF7A
:100BFE00FFFE07FFFFFFFFFFFFFFEAFFFFFC0FFFF8
:100C0E00FFFFFFAFFFFFF0FFFFFC17FFFFFFFF7FB0
:100C1E00FFFFFA7FFFF9EFFFFFFFFFEFFFFFFC7F04
:100C2E00FFF7EFFFFFFFFEFFFFFFFD1FFFF7EFFFD9
:100C3E00FFFF9FEFFFFFFE5FFFEFEFFFFFFC1DFFCC
:100C4E00FFFFFF0FFFEFFFFFFFE01FEFFFFFFF4F65
:100C5E00FFEFDFFFFC003FFFFFFFFF97FFDF02FF0D
:100C6E00F0003BEFFFFFFFC7FFDEEA3F80007FFF94
:100C7E00FFBFFFFFFFBFFFC8F800F7EFFF9FFFFFAB
:100C8E00FF7FFFEFF801FFFFFF03FFFFFF7FFFFF77
:100C9E00FE03EFEFFF51FFFFFEFFFFFFFF07FFFF1A
:100CAE00FFC47FFFFEFFFFFFFF9FEFEFFFF11FFF70
:100CBE00FDFFFFFFFD7FDFFFFFFC47FFFDBFFFFFD7
:100CCE00EEFBFFEFFFFF13FFFB5FFFFD73FBDFEF9D
:100CDE00FFFFC1FFFB1FFFFC8FFDBFEFFFFFF7FF05
:100CEE00F69FFFFA3FFDFFDFFFFFFBFFEB5FF1FE1D
:100CFE00FFF7BF6FFFFFFFFFE97FEEFCFFFDFFDF9A
:100D0E00FFFFFFFFF1FFFFFEFFF77EEFFFFFFFFF8D
:100D1E00DDFFFE7AFFFEFDAFFFFFFFFFEFDFF83EC8
:100D2E00FFF7FBDFFFFFFFFFAFE0FCBAFFF7F6AF09
:100D3E00FFFFF9FFA7E7FFCEFFFFDFEFFFFFE5FFA6
:100D4E00F3F8FFB6FFF7F56FFFFF01FFBBF5FF7A74
:100D5E00FFFFAFAFFFF82BFFBDF5FF7EFFFF7AEF72
:100D6E00FFE48FFFFAFBFEF5FFEFDF6FFF017FFF62
:100D7E00BCBBFEFAFEFF215FFF55FFFFBE7FFEF9F3
:100D8E00FEEFBFFFFF0FFFFFBA2FFEFBFF7EBFFF81
:100D9E00FFBFFFFFFF75FDB9FEEFBFFFFFFFFFFFB8
:100DAE007D5EFDFDFFBEFFFFFFFFFFFFFEFFFD7E31
:100DBE00FEEF7FFFFFFFFFFF7EBFFDFDFFDF7FFF2B
:100DCE00FFFFFFFFFF7FFDBDFEEEFFFFFFFFFFFFFB
:100DDE007FFFFB7FFFFF7FFFFFFFFFFF7FFFFDD644
:100DEE007EFD7FFFFFFFFFFFFFFFFD7ABFFF7FFF4F
:100DFE00FFFFFFFFBFFFFDDEDFF57FFFFFFFFFFF02
:100E0E00CBFFFE6BAEEB7FFFFFFFFFFFFBFFFF9EF7
:100E1E00F7EEFFFFFFFFFFFFFBFFFFF7BBDFFFFF5D
:100E2E00FFFFFFFFFBFFFFFFECEFFFFFFFFFFFFFEB
:100E3E00FBFFFFFFF6BFFFFFFFFFFFFFFFFFFFFF01
:100E4E00FCDFFFFFFFFFFFFFFBFFFFFFF75FFFFF73
:100E5E00FFFFFFFFFBFFFFFFFD3FFFFFFFFFFFFF5A
:100E6E00FFFFFFFFFF7FFFFFFFFFFFFFFBFFFFFF08
:100E7E00FD7FFFFFFFFFFFFFFFFFFFFFFF7FFFFF76
:100E8E00FFFFFFFFFFFFF7FFFD7FFFFF0101303187
:100E9E003233343536373839414243444546000003
:00000001FF
